:020000040000FA
:020000000428D2
:08000800FF30A200FF30A3004D
:100010008920AF200030D0200030DC20A501A601CF
:10002000A701A801A901AA01AB01A010A901FF30F5
:10003000AC00342024102608290203182028241498
:10004000CF20A4102708290203182728A414CE20A3
:1000500024112808290203182E282415CD20A90AC6
:10006000AC0B1928162833288E202D08AB00201D34
:100070003B28A0143C28A010A01C65282B08AD002C
:1000800081202E08A5002F08A600A010A01C49283A
:1000900052288E202D08AB00201D5028A014512876
:1000A000A01046282B08AD0081202E08A7002F089D
:1000B000A800AD0126086620A600AD01270866202D
:1000C000A700AD0128086620A8000800AE00003097
:1000D0002D078A000208053E2E0703188A0A8200AF
:1000E00000340134023403340434063409340D344A
:1000F00013341B3428343A3454347A34B034FF3453
:100100000800AF002D0E0F39AE002D080F39AF00DB
:10011000080003309F00ED201F13F02898189C283A
:100120001819A6288C1EAC288B138B1B94281A0830
:100130008B172015AD0008008B138B1B9C28181201
:100140001A081A081A0818168B178E288B138B1B7F
:10015000A6281A088B178E282011080008002311E2
:10016000E520A314E620ED20181398161812181590
:100170001810181DBE280C309900C2281819C22862
:1001800002309900F02098171813181618111A0841
:100190001A081A08003099000800D928D928D92847
:1001A000A50025080F39A6002408F0392604A4006C
:1001B000D928240885000800A50025080F39A600C5
:1001C0002208F0392604A200EA28E728E7282308B5
:1001D0006600080022086500080083160313080063
:0601E00083120313080066
:02400E00103F61
:00000001FF
